S01700006F70656E626C745F786D63313430302E73726563AD
S31510001000002000205D2A00100000000000000000F3
S31510001010001804000001000080B500F0C8FAC007EF
S31510001020C00F02BD0020C0435A4908605A490860E3
S31510001030704770B504000D00160000F059F9FF282E
S3151000104005D06019401E00F053F9FF2801D1002089
S3151000105070BD200A00025149884206D12B00320089
S3151000106021004D4800F09EF870BD2B003200210083
S31510001070484800F097F870BD70B504000E0000F0F7
S3151000108037F90500A019401E00F032F9FF2D01D0E6
S31510001090FF2801D1002070BD0100280000F0EDF8F6
S315100010A070BD80B53C4801680022D243914201D1FF
S315100010B0012002BD416882688918C26889180269D0
S315100010C089184269891880690818C143491C00911A
S315100010D06A4604213248FFF7ACFF02BD2F4801686B
S315100010E04268891882688918C2688918026989183D
S315100010F04269891880690818401E8041C00F7047E0
S3151000110010B50024E44324480168A14203D000F03E
S3151000111084F8002807D01F480168A14205D000F0C6
S315100011207CF8002801D1002010BD012010BD1B48FD
S31510001130704780B50A0601D0002002BD02688A42B7
S3151000114001D1012002BD016080225200001D00F075
S3151000115075FA012002BD38B505000C000E4885420F
S3151000116008D10C4D21002800FFF7E3FF00280DD110
S31510001170002032BD09498C4201D10500F2E7280052
S3151000118000F04BF80028EDD1002032BD280032BD0A
S3151000119000000000D8010020DC0200200030001002
S315100011A018300010F4B582B004000D001F00280A94
S315100011B00002009020680021C943884205D1009999
S315100011C02000FFF7B6FF00281CD02068009988423F
S315100011D004D02000FFF7BFFF040013D02068281AA0
S315100011E02018061D029D00F03DFA80204000211DAA
S315100011F0711A814209D3009909182000FFF7ABFF35
S31510001200040001D10020FEBD261D28783070761C02
S315100012106D1C7F1EE7D10120FEBD38B50400206885
S3151000122000F066F8FF2824D000F0BAF900F038FA7A
S3151000123005006D1D211D206800F0E3F905E000F0A2
S315100012402FFA854215D300F00DFAFFF7E5FE0028B8
S31510001250F5D100F0ACF900280BD1002000E0401CBD
S31510001260FF2808D82168091809782218127991429E
S31510001270F5D0002032BD012032BDF8B50F000200B6
S31510001280914230D3010003292DD3390033292AD2B4
S31510001290040000E0641C38002100C9B2884224D33F
S315100012A000F0E0F92000C0B200F03CF80500002084
S315100012B0C043854217D000F073F900F0F1F906002B
S315100012C00A36280000F098F905E000F0E9F98642A0
S315100012D009D300F0C7F9FFF79FFE0028F5D100F0FB
S315100012E066F90028D6D00020F2BD0120F2BD00001C
S315100012F038B50400002501E06D1CEDB2302D0FD27B
S3151000130000F0B0F913A06900491989004018016866
S315100013108C42F1D3426889188C42EDD2007A32BDE4
S31510001320FF2032BD70B504000025ED43002600E015
S31510001330761CF6B2302E0BD200F094F905A071008F
S31510001340891989004018017A22009142F0D1056866
S31510001350280070BD003000100010000003000000CF
S3151000136000400010001000000400000000500010A3
S3151000137000100000050000000060001000100000C2
S3151000138006000000007000100010000007000000AA
S3151000139000800010001000000800000000900010EF
S315100013A0001000000900000000A00010001000004E
S315100013B00A00000000B00010001000000B00000032
S315100013C000C00010001000000C00000000D000103B
S315100013D0001000000D00000000E0001000100000DA
S315100013E00E00000000F00010001000000F000000BA
S315100013F00000011000100000100000000010011085
S315100014000010000011000000002001100010000064
S315100014101200000000300110001000001300000040
S3151000142000400110001000001400000000500110D0
S3151000143000100000150000000060011000100000F0
S3151000144016000000007001100010000017000000C8
S31510001450008001100010000018000000009001101C
S31510001460001000001900000000A00110001000007C
S315100014701A00000000B00110001000001B00000050
S3151000148000C00110001000001C00000000D0011068
S31510001490001000001D00000000E001100010000008
S315100014A01E00000000F00110001000001F000000D8
S315100014B000000210001000002000000000100210B2
S315100014C00010000021000000002002100010000093
S315100014D0220000000030021000100000230000005F
S315100014E000400210001000002400000000500210FE
S315100014F0001000002500000000600210001000001F
S3151000150026000000007002100010000027000000E6
S315100015100080021000100000280000000090021049
S31510001520001000002900000000A0021000100000AA
S315100015302A00000000B00210001000002B0000006E
S3151000154000C00210001000002C00000000D0021095
S31510001550001000002D00000000E002100010000036
S315100015602E00000000F00210001000002F000000F6
S3151000157000000310001000003000000000100310DF
S3151000158000100000310000000020031000100000C1
S315100015903200000080B500F00AF8C007C00F02BD87
S315100015A013480188C02292010A43028070471148ED
S315100015B00088704780B50A00010010008222520090
S315100015C01268904701BD70B505000C0000260CE0AE
S315100015D028008021490009688847FFF7DBFF0028AB
S315100015E0FBD1802040002D18761CA642F0D370BD8A
S315100015F0040005400000054080B51021FFF7E3FF09
S3151000160001BD80B5FFF7D6FF01BD80B500F054F8D7
S3151000161001BD10B500F060F800280ED000F06EF88D
S3151000162000280AD000F09CF800F02DF800F058F8C9
S31510001630001D046800F042F8A04710BD70B51400F4
S315100016400D00060005E0287830706D1C761C00F041
S3151000165009F82000441E0004F5D170BD80B500F0D5
S3151000166052F801BD80B500F053F801BD80B500F009
S315100016700AF80E480E494160002181600522026079
S315100016800C48016001BD00200849086070470748F2
S315100016900068C00303D507480168491C01607047FC
S315100016A080B5FFF7F4FF0348006802BD10E000E0C4
S315100016B07FBB0000B004002072B6704762B6704758
S315100016C080B5FFF7AFFC01BD80B5FFF7B2FC02BDD8
S315100016D080B5FFF7D1FC02BD80B5FFF7FFFC02BD58
S315100016E080B5FFF724FD02BD80B5FFF7DAFC0028B0
S315100016F001D1002002BDFFF703FD02BD80B500F049
S3151000170099F8012002BD80B5642000F066F801BD8D
S3151000171080B500F072F801BD10B500F097F800F032
S3151000172083FA294C0120207000F07AFB00202070EB
S3151000173010BD10B5244C201D00F017FB012804D154
S3151000174001202070201D00F09CF8201D00F0B4FB35
S31510001750012804D100202070201D00F092F810BD41
S31510001760704770B506000C00174D2878012803D174
S31510001770C9B2300000F0D9FA2878002804D1210027
S31510001780C9B2300000F070FB00F077F870BD0E485B
S315100017900078401E03D0401E012802D903E008201D
S315100017A07047002070474020704707480078401E59
S315100017B003D0401E012802D903E0082070470020FC
S315100017C070474020704700008001002080B500F06F
S315100017D04DF802BD8A404260704738B50400194D75
S315100017E080220021280000F0EFFB012200212800B2
S315100017F0FFF7F0FF1448448031BD10B5FFF750FFD6
S31510001800114C6168884214D30E482178002906D1FC
S31510001810012121700A040021FFF7DCFF04E00021FA
S3151000182021700122FFF7D6FFFFF73AFF61884018B3
S31510001830606010BD80B5012200210248FFF7CAFF83
S3151000184001BD000000040440A004002010B40020D4
S31510001850BB4902000A800A00443250600300432448
S315100018600B55138002008A7010BC7047B44801787B
S31510001870481E8041C043C00F70470020B149087010
S31510001880704710B50178AE4CFF2913D100F081F8DE
S315100018904320205C012802D1102000F071F844206A
S315100018A0215E012905DB01204322A054E01C00F033
S315100018B04FF810BD2278012AFBD1C92932D0CC2984
S315100018C03FD0CF293AD0D0292FD0D12933D0D22901
S315100018D02ED0F32917D0F4290FD0F5290AD0F629DE
S315100018E00ED0FA2912D0FC2913D0FD2914D0FE29C6
S315100018F015D029E000F0A6F8CAE700F0C0F8C7E74F
S3151000190000F097F8C4E700F0D9F8C1E700F080F8C6
S31510001910BEE700F077F8BBE700F065F8B8E700F02F
S3151000192056F8B5E700F0EFF8B2E700F00DF9AFE7BB
S3151000193000F0D7F8ACE700F034F9A9E700F044F965
S31510001940A6E700F04DF9A3E7202000F019F89FE76D
S3151000195080B589B2FFF705FF01BD10B4002303E07F
S3151000196004781B19DBB2401C0C00611E002CF7D149
S315100019701360012010BC70470020714948707047F1
S315100019806F49CA1CFE2313705070022044228852DD
S31510001990704738B5FFF7F0FF694C01252570FF2019
S315100019A0E0701020207100206071FFF7F0FEA0712A
S315100019B0FFF7FBFEE071FFF7F8FE000A2072657272
S315100019C0A572082044216052FFF77AFE31BD10B58A
S315100019D05B4C00202070FFF7CFFFFF20E070012046
S315100019E04421605210BD5648411CFF228A700022C5
S315100019F0CA700B780B714A718A71CA71062144221A
S31510001A008152704780B50020FFF7BAFF01BD000074
S31510001A104B48C11CFF220A70443000BF73A24260BB
S31510001A2000224A708A70CA7007224A600821018013
S31510001A3070474349FF22CA7044314068486001200C
S31510001A400880704770B50500FFF7A1FE6A78401E42
S31510001A50904203DA2220FFF793FF70BD384C260020
S31510001A6044367168201DFFF7E9FDFF20E0707068AD
S31510001A706978401870606878401C308070BD70B509
S31510001A800400FFF784FE401E6178884203DA2220A4
S31510001A90FFF776FF70BD6168294D2E0044367160E0
S31510001AA06278281DFFF7CAFDFF20E870706861781C
S31510001AB0401870606078401C308070BD38B5204981
S31510001AC0CC1CFF2222700D004435CA1D416868687F
S31510001AD0FFF743FF60700020A070E0700820288098
S31510001AE031BD70B5164CE51CFF20287000266E70AF
S31510001AF0AE70FFF74CFEE8702E716E71AE71072056
S31510001B004421605270BD70B50600FFF740FE0C4CC4
S31510001B1025004435721C411E6868FFF7D5FD002864
S31510001B2003D13120FFF72CFF70BDFF20E070FFF7C7
S31510001B302EFE6968401E081868600120288070BD56
S31510001B402C0400206F04002038B50400FFF71FFE98
S31510001B50801E6178884203DA2220FFF711FF31BD1B
S31510001B601E48FF21C1700500443501202880617888
S31510001B70080007D1FFF7B8FD002811D13120FFF773
S31510001B80FFFE31BDA21C6868FFF79EFD002803D139
S31510001B903120FFF7F5FE31BD68686178401868603E
S31510001BA031BD38B50D4C2500443541686868FFF7DE
S31510001BB08FFD002803D13120FFF7E2FE31BDFF2053
S31510001BC0E0700120288031BD80B5FFF722FD034863
S31510001BD0FF21C17001214422815201BD2C04002035
S31510001BE080B53120FFF7CCFE01BD00004F70656E49
S31510001BF0424C5400016840220A4302607047016853
S31510001C004022914301607047016801220A43026035
S31510001C107047016801229143016070470068C069EE
S31510001C2070470068C1617047FEB500F0FBF904000B
S31510001C305E4800E064008442FCD35D48844201D3D0
S31510001C406408FAE7220001215A4800F0D3FA0094FA
S31510001C50594801906846FA214901018101264681B9
S31510001C60564C6946606A00F00BFA606AFFF7C2FFCD
S31510001C70606AFFF7C9FF52482060770761683940EC
S31510001C80504808436060A1684A0F52074E491143F5
S31510001C90A1604E4A024062603943A1600820207359
S31510001CA00025280003E0C0B221180D74401C010065
S31510001CB0227BC9B29142F6D32676200000F0F5FABF
S31510001CC02A4631463B4800F065FA41483C492031E6
S31510001CD0016042683A403F49114341608268530FA0
S31510001CE05B073D4A1A438260384B0B4043601743EB
S31510001CF0876008210173290003E0C9B242181574E0
S31510001D00491C0A00037BD2B29A42F6D3057600F03C
S31510001D10CCFA32461146274800F03CFA606AFFF7C3
S31510001D206EFF606AFFF775FFF7BD10B5234C217380
S31510001D30002104E0425C63181A74491CC9B2227B64
S31510001D409142F7DB200000F0F7FA02212000FFF79E
S31510001D5068FF200000F011FB01E0FFF783FC200074
S31510001D60FFF75CFF8007F8D410BDF1B500263400EC
S31510001D700127174D2800FFF751FF384013D02800D0
S31510001D8000F010FB00280AD106E0A819007C009983
S31510001D9088553C00761CF6B2287B8642F5DB394620
S31510001DA02800FFF73EFF2000F2BD0000001BB70021
S31510001DB0010E27070000045020A10700580100203B
S31510001DC000100450E1070080E1070000FFFFFFDF6D
S31510001DD07804002067060080670600008A21490003
S31510001DE04058010B0800C007C00F70478A214900F0
S31510001DF04158C0208000084070478C225200815004
S31510001E0070478A2149004058C1080800C007C00F12
S31510001E107047016C0F22914302220A4302647047F5
S31510001E2010B584B0E1200002009008206946020037
S31510001E300A714871012088711020C871002008812C
S31510001E40504C606800F0E8FA012304221021606803
S31510001E5000F0EAFB012304220021606800F0F7FB82
S31510001E606068FFF7D6FF1FBD70B506000C00412C49
S31510001E7003DB752145A000F025FC200000F065F875
S31510001E80012804D0792100BF40A000F01BFC0025DA
S31510001E900CE0FFF7E7FBADB2705D00F056F80128D5
S31510001EA003D0822139A000F00DFC6D1C2800210002
S31510001EB080B28842EDD370BD38B50500324C6078DB
S31510001EC000280FD1201D00F02FF801282AD12079E3
S31510001ED0002827D0FFF7E4FBA06400202070012023
S31510001EE060701FE020782018401D00F01DF80128B2
S31510001EF010D12278521C227010002179C0B288426B
S31510001F0010D1D2B2611D2800FFF798FB0020607037
S31510001F10012032BDFFF7C4FBA16C6431814201D2AE
S31510001F2000206070002032BD38B5040015484568A1
S31510001F302800FFF766FF002805D1280000F0C2FA36
S31510001F402070012032BD002032BD70B506000D4C48
S31510001F5065682800FFF742FF002801D0002070BDF9
S31510001F603100280000F094FA802676006568280073
S31510001F70FFF73CFF3040F9D031002800FFF73DFF56
S31510001F80012070BDC4010020E0030020433A5C57D5
S31510001F906F726B5C736F6674776172655C4F706598
S31510001FA06E424C545C5461726765745C536F757203
S31510001FB063655C41524D434D305F584D43315C75FE
S31510001FC06172742E6300000010B48B089B00C01859
S31510001FD0CB00182119400369FC248C40A3430361EC
S31510001FE003698A401A43026110BC7047C3200C492A
S31510001FF0086070470A48C021016001684907FCD48F
S31510002000704710B50400FFF7F5FF084801690C4347
S31510002010046101684900FCD4FFF7E8FF10BD000019
S315100020202400014002480068704700000003014088
S31510002030D4010020E22149004058C0218900014006
S31510002040481E8041C00F704712040A4319061143F7
S31510002050E222520081507047016840220A43026012
S3151000206070470168402291430160704702000800E2
S31510002070904200D210007047884200D9080070477D
S31510002080F3B587B0002005900121029101907E489A
S3151000209004900C460A2600E0641C412C3BD208989A
S315100020A00068810008184000210000F00FFB0500B1
S315100020B00898406800902800009900F007FB0390EC
S315100020C0310000F003FB07000398310000F005FB18
S315100020D0062900D37F1C002F06D02800B900C91985
S315100020E0490000F0F3FA04E02800310000F0EEFA9F
S315100020F001270099884201D3401A00E0081A152FCB
S31510002100CAD204998842C7D2059401970490FA213D
S3151000211089008842C0D25C4C402500E06D1E032D1C
S3151000212013D32800401C58494843019900F0CEFAB1
S3151000213008990989884201D3421A00E00A1AA24274
S3151000214001D2029514008842E8D20798FFF784FF5F
S3151000215001980299401A801E0003E021C90101402E
S3151000216008984089401E8001C02202400A43029806
S31510002170401E0002F0210901014011430598401E3E
S315100021808006800E0843079908610798FFF769FFD4
S3151000219009B0F0BD70B504000D0016002000FFF761
S315100021A049FF0028FAD06D1C2B00DBB23200022149
S315100021B02000FFF749FF70BD10B504008020800392
S315100021C0FFF71FFF206801218843206020688007E1
S315100021D0FCD410BD80B500F062F8012802D00228A8
S315100021E003D005E0FFF71EFF02BD00F085FA02BD21
S315100021F0002002BDF0B583B004000E001500FFF7F5
S31510002200DBFF3100200000F041F82000FFF7E2FF6D
S3151000221000908026F600290000F058FA311A0020A6
S31510002220FFF724FF761E3100FFF726FF0190009876
S315100022308709A8098002390000F048FA3100FFF733
S315100022401BFF060000988021C900019A891A00F028
S315100022503DFA281A7743B90A8901691A81428041E1
S31510002260C043C00F03D0019E01D0012000E0022020
S31510002270E168604A0A40E260E168800306430E4363
S31510002280E660F7BD0000000010270000E4225200AF
S31510002290801802680F239A43114301607047E421A6
S315100022A0490040580007000F704738B504002168F0
S315100022B05148081840098A68504B13408B602168B2
S315100022C08A6843095B030002F8256D0105401D432A
S315100022D015438D60207E010001D001282BD12020CE
S315100022E02168C8616068216802009200D20F0CD183
S315100022F0420F5207800410438861A068410F4907B6
S31510002300800408432168C86003E08861A0682168DA
S31510002310C860207E012807D1200000F00DF880202B
S3151000232000052168C86103E0802000012168C861AA
S3151000233033482168C86131BD010003200A7E012A95
S3151000234000D0704710B420200A68D061086802686F
S315100023502C4B13400A7B1206F024240514401C4310
S31510002360046008690A68106148690A68506126485D
S315100023700968C861002010BC704700680121C26955
S3151000238052090A40C3691B0A1940002A01D10420C8
S315100023907047012901D102207047E021C904C161AB
S315100023A00020704710B402680121D369DB0A0B4084
S315100023B0D26992080A40002B01D0032017E0012AA7
S315100023C001D1022013E002681269026102685269A3
S315100023D042610268D3699C080B002340D269D40875
S315100023E00A002240002B01D0002AECD1002010BC9C
S315100023F070470000003CFFFF00F0FBAFFF00FFFF3F
S315100024004000A006FFFFFFF040002800806B8021EF
S3151000241008407047C164704770B504000E0010255F
S3151000242000F09CF8F079010000D005002A00316810
S31510002430200000F0B3F8B079401E4000AD1CE90151
S31510002440FF229143014311480843E0633079401E4F
S315100024500006D11C014361637079010005D0616BE0
S31510002460401E00040843606305E0606B3179491E25
S31510002470090401436163A020C000A0630020C0438B
S31510002480E0640820305E206470BD00000100030087
S3151000249038B504000D008420400020180168E022A1
S315100024A0D2040A400CD12000FFF7B0FF8028FAD0E2
S315100024B0802189012000FFF7ADFF8020255031BD16
S315100024C0856731BD8621490041180A68E023DB047F
S315100024D0134001D1406D00E0086980B27047F8B42E
S315100024E00168421843685908511800918168DB0742
S315100024F001D54B46C918009B9A4202D10C30F2BC4A
S3151000250070471378521C032403261E4002D11678F6
S31510002510F61C521C1D090F2D07D115780F35521CAC
S3151000252003E01778521C0F70491C761EF9D1002D46
S31510002530E1D01678521C9B081C40032C01D114784C
S31510002540521C2302F3185C420B19AD1CD3D01C7815
S315100025505B1C0C70491C6D1ECDD0F8E710B504003D
S315100025609020C005844202D04C48844203D14C4886
S3151000257000F083F808E04B48844202D04A4884426F
S3151000258002D14A4800F079F80320E060E068C007FD
S31510002590FCD5206C0F218843206410BDF1B584B0A2
S315100025A00D001400642D3CD3002C3AD06426FFF79E
S315100025B039FD310000F08AF802902800310000F051
S315100025C085F8050001260196394F0097002F13E074
S315100025D0029878432900614300F078F8810A800553
S315100025E0800D8022D200914205D2009A904202D2EA
S315100025F000900E0001977F1EEAD1019880210902F2
S31510002600014304980161049840692A490140641EF7
S31510002610A0020843761E310401430498416100204C
S3151000262000E0012005B0F0BD30B484246400001928
S315100026300468214D254005600468204D25401B0285
S315100026402B43194312060A43026030BC704730B45C
S315100026508624640000190468174D25400560046837
S31510002660174D25401B022B43194312060A4380219E
S3151000267049051143016030BC704780B5084988424E
S3151000268003D10820FFF7BDFC01BD0849884203D1DC
S315100026908020C002FFF7B5FC01BD00000002004813
S315100026A00800004800400048004200480840004822
S315100026B0FF030000EF8000FCFFFFFFF8C0C0FFF82B
S315100026C0C0C0FFEF80B5FEF7CDFFFCE7094A042333
S315100026D05361106051609068704710B4054C042225
S315100026E0626120606160E2681300A06800211943EE
S315100026F010BC70472000034000487047002D310180
S3151000270089004018C169072399430A43C26170477B
S3151000271038B58B00C318DC695025AC43DC61FFF774
S31510002720EFFF31BDC26807239A434907490F11438A
S31510002730C1607047016840220A4302607047016811
S31510002740402291430160704780B500F007F800F011
S3151000275043F800F004F800F04DF8FCE7704730B588
S3151000276089B0002468460476174D06AA032128006E
S3151000277000F04AF89C206946087404AA0221280031
S3151000278000F042F8224611461048FFF7C1FF68468E
S3151000279004720F4C02AA0821200000F035F8A4207C
S315100027A0694608706A460921200000F02DF8094C88
S315100027B02000FFF7BFFF02212000FFF7B3FF200024
S315100027C0FFF7BDFF09B030BD00010440000200480C
S315100027D0000404400003045080B5FEF716FFFEF710
S315100027E03DFFFEF743FFFEF76BFFFEF795FF00F088
S315100027F04FF801BD80B5FEF735FFFEF748FFFEF72F
S3151000280098FF00F04FF801BDF8B40B000324A34362
S31510002810C318CD0018242C401D69FC26A640B543CC
S315100028201D61456F03264F00BE40B5434567CD0871
S31510002830AD0045196F46BC468F001C263E406746C4
S315100028403E702E6CB44604276E463678B740664600
S31510002850BE432E642E6CB44657786E463678B74013
S31510002860664637432F64094DA84205D160352E6858
S3151000287001278F40BE432E6055688D40456018690C
S315100028801178A14001431961F1BC70470002044060
S3151000289010B50F4C01202070FEF702FF606000F0AB
S315100028A001F810BD10B5FEF791FF01280FD0084CA6
S315100028B0207801280BD1FEF7F3FE6168FA22520048
S315100028C08918884203D300202070FEF7A2FE10BD9F
S315100028D098040020F8B519480168090ACAB2184BBD
S315100028E01A60184C410D002A1ED00568EDB25D60C5
S315100028F0C6693702C026B6003E402E435E6092027D
S315100029009519C069014006D10F482900FFF7DEFE70
S3151000291000012060F1BDFFF7EFFE80012900FFF7EF
S31510002920D5FE00012060F1BDC069014002D1074803
S315100029302060F1BDFFF7E0FE2060F1BD000301400D
S31510002940A8040020D401002000001BB7006CDC0294
S3151000295070B40121002213E00468001D0C4202D05D
S315100029604D466D1E64192260241D1B1F042BFAD2BE
S3151000297025009E0701D52280AD1C0B4000D02A7081
S315100029800368001D002BE7D170BC704780B507485F
S31510002990C02101600649CA69064B1340CB61064A3D
S315100029A00A60C3210160FFF795FF01BD24000140B5
S315100029B000030140FFFDFFFF0001F13F10B507497D
S315100029C079441831064C7C44163404E0081D0A6814
S315100029D0891888470100A142F8D110BD08000000EF
S315100029E0340000006DFFFFFFDC020000D80100205C
S315100029F000000000EBFAFFFF0901000026010000AD
S31510002A000C000020DBFAFFFFDA0000003E00000099
S31510002A105801002000F00BF8002801D0FFF7CEFF78
S31510002A20002000BF00BFFFF78FFE00F002F8012064
S31510002A30704780B500F002F801BDFEE7074638463C
S31510002A4000F002F8FBE7FEE780B500BF00BF024AC0
S31510002A5011001820ABBEFBE726000200024885468F
S31510002A60024880470248004700200020852A0010AF
S31510002A70912A0010024801680122914301607047B3
S31510002A806800014080B5FFF7F5FFFFF77FFF01BD36
S31510002A9000BF00BF00BF00BFFFF7BCFFFEE7FEE7A9
S31510002AA0FEE7FEE7FEE7FEE7FEE7FEE7FEE7FEE7E8
S31510002AB0FEE7FEE7FEE7FEE7FEE7FEE7FEE7FEE7D8
S31510002AC0FEE7FEE7FEE7FEE7FEE7FEE7FEE7FEE7C8
S31510002AD0FEE7FEE7FEE7FEE7FEE7FEE7FEE7FEE7B8
S31510002AE0FEE7F20F0001F007340204500003045011
S31510002AF004000110014800020412400400014200C3
S31510002B004820022C48004704122B04122A041229CA
S31510002B1004122804122704522604122404522308ED
S31510002B20F173041003472A00103B04129D04129FF0
S31510002B300412A10412A30412A50412A70412A904D4
S31510002B4012AB0412AD0412AF0412B10412B3041284
S31510002B50B50412B70412B90412BB0412BD0412BF95
S31510002B600412C10412C30412C50412C70412C90404
S31510002B7012CB0412CD0412CF0412D10412D30412B4
S31510002B80D50412D70412D90412DB0412DD0412DFA5
S30910002B900412E10430
S70510002A912F
